:1000000012C00CC129C028C027C061C025C024C0AF
:1000100023C022C021C020C01FC01EC01DC01CC0E4
:100020001BC01AC019C011241FBECFEDCDBF10E0F8
:10003000A0E6B0E0E6EFF2E003C0C89531960D927D
:10004000AE3BB107D1F710E0AEEBB0E001C01D92BE
:10005000A63CB107E1F70BC1D3CFCF93DF93CDB768
:10006000DEB7AFE5B0E0EFE5F0E0808180688C932B
:10007000DF91CF910895CF93DF93CDB7DEB7AFE592
:10008000B0E0EFE5F0E090818FE789238C93DF917A
:10009000CF910895CF93DF93CDB7DEB7ECE4F0E0D6
:1000A0008091BC009091BD0091838083EFE4F0E0EB
:1000B0001082EEE4F0E081E08083E2E4F0E0108280
:1000C000E9E5F0E080E88083DF91CF9108951F9209
:1000D0000F920FB60F9211242F933F935F936F935C
:1000E0007F938F939F93AF93BF93EF93FF93CF93A0
:1000F000DF93CDB7DEB7ECE4F0E08091BC009091E7
:10010000BD00918380838091BE009091BF002091BB
:10011000C0003091C100732F622FD7D02091B8005A
:100120003091B900732F622FBED02091C000309162
:10013000C100732F622FC9D0972F862F282F392FF8
:100140008091C2009091C300820F931F9093C500CD
:100150008093C4002091C4003091C5008091BA0002
:100160009091BB002817390768F4A8E3B0E08091AC
:10017000C4009091C500F92FE82FE05AFF4F80810D
:100180008C931CC02091BA003091BB008091B800C4
:100190009091B900280F391F8091C4009091C5003B
:1001A0008217930720F4E8E3F0E0108207C0E8E349
:1001B000F0E010821092C3001092C2008091BE0045
:1001C0009091BF0001969093BF008093BE00DF9195
:1001D000CF91FF91EF91BF91AF919F918F917F91BF
:1001E0006F915F913F912F910F900FBE0F901F90D5
:1001F0001895CF93DF93CDB7DEB7A5E5B0E0E5E581
:10020000F0E0808183608C93ABE5B0E0EBE5F0E05B
:10021000808180648C93DF91CF9108951F920F921B
:100220000FB60F9211248F939F93CF93DF93CDB787
:10023000DEB78091BE009091BF009093C100809383
:10024000C0001092BF001092BE008091C200909139
:10025000C30001969093C3008093C200DF91CF91B9
:100260009F918F910F900FBE0F901F901895CF9375
:10027000DF93CDB7DEB7E7E3F0E08081E7E3F0E0BE
:100280008FEF8083E8E3F0E08081E8E3F0E0108224
:10029000A2E3B0E0E2E3F0E0808184608C93FADED8
:1002A000A8DFDBDEFFCF5527002480FF02C0060E4B
:1002B000571F660F771F6115710521F09695879579
:1002C000009799F7952F802D0895AA1BBB1B51E12C
:1002D00007C0AA1FBB1FA617B70710F0A61BB70BB6
:1002E000881F991F5A95A9F780959095682F792FA7
:0602F0008A2F9B2F0895E8
:1002F6000000000000000000542A0108010801085F
:10030600542A0000000000000000142241084108A1
:100316004108552A000000000000000000224100AC
:1003260041004100142A00000000000000000814EB
:10033600002241004100552A000000000000000094
:0E034600410041084108552A40005800E0FCE3
:00000001FF
